:020000040000FA
:10000000B6017029B616B61EB612B6190B28B6156B
:100010004420031832280830A3005820A20DA30B57
:100020000D28B61E3D2062205E20B61A32203720F1
:10003000220803106B29B616B61EB61236192528EB
:10004000FE39B700361503106B29361A2D28A60085
:10005000361644200318322826084B20031832286D
:10006000B61E6B293D20622036113612B6113A08B1
:10007000840038088417800443283A08840038092B
:100080008005841780050800372062203D205E200F
:100090003708B6190138A2000830A300A20D0318D2
:1000A0003720031C3D2062205E20A30B4E28372002
:1000B00062203A08840038080005FF3E3B088400AF
:1000C000390940283B08840039083A280408A70069
:1000D0000612861286128316061286128612F030D7
:1000E000860583122708B61893283A30A100983065
:1000F00009213330A600A8201330A100883009213F
:10010000A82064300821A820643008212230A600ED
:10011000A820283092200C30922006309220B6146D
:10012000270893283614A600361CA1288612033C03
:10013000031CA628A6200730A100D03009210314F3
:1001400008003614FE3C03196B298616A60E361CD1
:1001500036100616F030860526080F39860406127A
:10016000A60E3618A8283230082103140800B71349
:1001700029080319B7170530A8002730A30010304D
:10018000CD200330A300E830CD20A3016430CD2082
:10019000A3010A30CD202408D428A2002508A100FC
:1001A0002408A00034212008A000A8030319B713D5
:1001B00029080319DE282802031808002008031D57
:1001C000B713B71B0800303E662903178D0083164E
:1001D0008C130C1483120C086B2903178C008316E4
:1001E0008C130C1555308D00AA308D008C148C1892
:1001F000F7280C116B29A301A200FF30A207031CF2
:10020000A307031C6B290330A100E6300921FD2858
:10021000A101FC3EA000A109031C1429FF3000002D
:10022000A00703180F29A0076400A10F0E290800DA
:10023000A101A301A20002301D29A8002308210268
:10024000031D242922082002043003180130031959
:1002500002302805031DFF306B290038031DFF30D5
:100260000405031DFF306B29A501A4011030A60071
:10027000210DA40DA50D2208A4022308031C230FA1
:10028000A50203184A292208A40723080318230FEC
:10029000A5070310A00DA10DA60B382920086B2976
:1002A0001030A800A101A001A70CA60C031C5E2918
:1002B0002208A00723080318230FA107A10CA00CF4
:1002C000A50CA40CA80B542924086B298400310820
:1002D0008A0030088200831303138312640008002D
:1002E000831607309F008312C001C801BE01C701F9
:1002F000BD01C601FE308A01672040308A016720B7
:100300001E308A016720FE308A01672041308A0151
:1003100067200C308A016720FE308A016720423056
:100320008A0167200C308A016720FE308A0167202D
:1003300043308A0167200E308A016720FE308A012F
:10034000672044308A01672011308A016720FE301F
:100350008A01672045308A01672015308A016720AD
:10036000FE308A01672046308A01672011308A01F9
:100370006720FE308A01672047308A0167200E30EF
:100380008A016720FE308A01672048308A01672091
:1003900001308A016720FE308A01672049308A01D6
:1003A00067201C308A016720FE308A0167204A30AE
:1003B0008A01672019308A016720FE308A01672090
:1003C0004B308A0167201C308A016720FE308A0189
:1003D00067204C308A0167201C308A016720FE307C
:1003E0008A0167204D308A0167201C308A0167200E
:1003F000FE308A0167204E308A0167201C308A0156
:100400006720FE308A0167204F308A0167201C3048
:100410008A016720FE308A01672050308A016720F8
:100420001F308A016720FE308A01672051308A011F
:10043000672013308A016720FE308A01672052301E
:100440008A0167201B308A016720FE308A016720FD
:1004500053308A0167201B308A016720FE308A01F1
:10046000672054308A0167201B308A016720FE30E4
:100470008A01672055308A0167201B308A01672076
:10048000FE308A01672056308A01672011308A01C8
:100490006720FE308A01672057308A0167201F30AD
:1004A0008A016720FE308A01672058308A01672060
:1004B0001F308A016720FE308A01672059308A0187
:1004C000672011308A016720FE308A0167205A3088
:1004D0008A01672015308A016720FE308A01672073
:1004E0005B308A0167201D308A016720FE308A0157
:1004F00067205C308A0167201B308A016720FE304C
:100500008A0167205D308A01672017308A016720E1
:10051000FE308A0167205E308A01672011308A012F
:100520006720FE308A0167205F308A0167201F3014
:100530008A016720FE308A01672060308A016720C7
:100540001F308A016720FE308A01672061308A01EE
:10055000672011308A016720FE308A0167206230EF
:100560008A0167201D308A016720FE308A016720DA
:1005700063308A01672011308A016720FE308A01CA
:10058000672064308A0167201D308A016720FE30B1
:100590008A01672065308A01672011308A0167204F
:1005A000FE308A01672066308A0167201F308A0189
:1005B0006720FE308A01672067308A0167201F307C
:1005C0008A016720FE308A01672068308A0167202F
:1005D0001F308A016720FE308A01672069308A0156
:1005E000672015308A016720FE308A0167206A3053
:1005F0008A01672015308A016720FE308A01672052
:100600006B308A01672011308A016720FE308A0131
:1006100067206C308A0167201D308A016720FE3018
:100620008A0167206D308A0167201D308A016720AA
:10063000FE308A0167206E308A0167201F308A01F0
:100640006720FE308A0167206F308A0167201F30E3
:100650008A016720FE308A01672070308A01672096
:100660001B308A016720FE308A01672071308A01C1
:10067000672000308A016720FE308A0167207230CF
:100680008A0167200A308A016720FE308A016720CC
:1006900073308A0167200A308A016720FE308A01A0
:1006A000672074308A01672000308A016720FE309D
:1006B0008A01672075308A01672011308A0167201E
:1006C000FE308A01672076308A0167200E308A0169
:1006D0006720FE308A01672077308A016720063064
:1006E0008A016720FE308A01672078308A016720FE
:1006F0001B308A016720FE308A01672079308A0129
:10070000672000308A016720FE308A0167207A3036
:100710008A01672002308A016720FE308A01672043
:100720007B308A0167201A308A016720FE308A01F7
:1007300067207C308A01672000308A016720FE3004
:100740008A0167207D308A01672011308A01672085
:10075000FE308A0167207E308A0167200E308A01D0
:100760006720FE308A0167207F308A0167200630CB
:100770008A016720FE308A01672001308A016720E4
:10078000FE308A01672080308A01672020308A018C
:10079000672056308A01672041308A016720523035
:1007A0008A01672047308A01672041308A0167202B
:1007B00020308A01672056308A01672049308A013B
:1007C00067204B308A01672054308A0167204F3000
:1007D0008A01672052308A016720FE308A01672033
:1007E000C0308A01672020308A01672020308A01CA
:1007F000672020308A01672020308A01672032304C
:100800008A01672030308A01672030308A016720F2
:1008100039308A016720FE308A01672090308A01D2
:10082000672020308A01672020308A01672020302D
:100830008A0167204F308A0167204E308A01672085
:1008400054308A0167204F308A0167205A308A016C
:1008500067204F308A016720FE308A016720D03040
:100860008A01672020308A01672020308A016720B2
:1008700020308A01672056308A01672045308A017E
:1008800067205A308A01672045308A01672052303C
:100890008A0167204C308A0167204F308A01672027
:1008A000C1016400053041028A110A120318792C33
:1008B000FE308A0167208F308A01672006308A0166
:1008C00067200130A300F4308A01FC20FE308A0149
:1008D00067208F308A01672007308A016720013046
:1008E000A300F4308A01FC20C10A8A110A12031DF8
:1008F000512C081083160810831288108316881054
:100900008312081183160811831288118316881127
:1009100083120711831607110A3083128A01E5201A
:10092000C20014308A01E520C4001E308A01E5208F
:10093000CC006400183042028A110A12031CA12C58
:10094000C20164003C3044028A110A12031CA92C23
:10095000C401640015304C028A110A12031CB12C28
:10096000CC0128308A01E520C30032308A01E5201D
:10097000C5003C308A01E520CD00640018304302F8
:100980008A110A12031CC52CC30164003C304502C5
:100990008A110A12031CCD2CC501640015304D02CA
:1009A0008A110A12031CD52CCD01FE308A01672062
:1009B00001308A016720FE308A016720DF308A011A
:1009C000672006308A0167208A150A12CA22FE3083
:1009D0008A016720C0308A0167204C308A01672075
:1009E00031308A0167203A308A0167200230A9003D
:1009F0004208A400A5016630B000B1018A01B72009
:100A00003A308A0167200230A9004408A400A501F9
:100A10006630B000B1018A01B72020308A0167201A
:100A200020308A0167205A308A01672031308A01DC
:100A300067203A308A0167200230A9004C08A400E0
:100A4000A5016630B000B1018A01B72027308A01C4
:100A50006720FE308A01672090308A0167204C3081
:100A60008A01672032308A0167203A308A01672084
:100A70000230A9004308A400A5016630B000B1010E
:100A80008A01B7203A308A0167200230A900450860
:100A9000A400A5016630B000B1018A01B720203062
:100AA0008A01672020308A0167205A308A01672036
:100AB00032308A0167203A308A0167200230A9006B
:100AC0004D08A400A5016630B000B1018A01B7202D
:100AD00027308A01672064008A110A12081B732DCF
:100AE0008A150A12B62364008A110A12881B7B2D0C
:100AF0008A110A12992564008A110A12881A832D14
:100B00008A110A125A2664008A110A12081A8B2DB9
:100B10008A110A12E7278A110A12CE258A110A12AF
:100B20001426FA308A01FB208A01DB2C63008A013B
:100B3000962DFE308A016720D0308A016720003070
:100B40008A01672007158316071183120330A3005B
:100B5000E8308A01FC2064008A110A12881BB32D38
:100B60008A110A12BB2D8A150A12CA22C8308A01BC
:100B7000FB208A01AB2DFE308A016720D0308A012C
:100B8000672020308A01672007118316071183121E
:100B90000330A300E8308A01FC20080064004C0800
:100BA000003C8A110A12031DD82D8A110A12132E35
:100BB0003D08A600A7010A30A200A3018A01502126
:100BC000B2002508B30046083207CE003E08A60052
:100BD000A7010A30A200A3018A015021B200250812
:100BE000B30047083207CF004208A0004E088A0130
:100BF0001821B2004408A0004F088A011821B4004F
:100C00003208840034088A012D21B400B500640044
:100C1000340835048A110A120319132E4C08CB002C
:100C20008A150A127721080064004D08003C8A11D9
:100C30000A12031D1E2E8A110A12592E3D08A60003
:100C4000A7010A30A200A3018A015021B2002508A1
:100C5000B30046083207CE003E08A600A7010A30BE
:100C6000A200A3018A015021B2002508B300470861
:100C70003207CF004308A0004E088A011821B200B5
:100C80004508A0004F088A011821B40032088400EA
:100C900034088A012D21B400B500640034083504FD
:100CA0008A110A120319592E4D08CB008A150A120F
:100CB00077210800FE308A01672001308A01672011
:100CC000FE308A01672080308A01672031308A0136
:100CD00067202E308A01672020308A0167205A3031
:100CE0008A0167204F308A0167204E308A016720D1
:100CF00041308A01672049308A01672044308A01E7
:100D000067204F308A0167203A308A016720FE3021
:100D10008A016720C0308A0167200230A9004C0890
:100D2000A400A5016630B000B1018A01B7202030CF
:100D30008A01672050308A01672045308A01672088
:100D400052308A01672043308A016720C8308A0107
:100D5000FB2064008A110A12881BAF2ECC0A6400A3
:100D600015304C028A110A12031CB72ECC01640004
:100D70008A110A12881ABF2E8A110A12C12E8A01FC
:100D8000872E03171E308D0003134C088A01ED20B7
:100D90000A308A01FB20FE308A01672001308A0177
:100DA0006720FE308A01672080308A016720313059
:100DB0008A0167202E308A0167204C308A01672023
:100DC0004F308A01672043308A01672053308A01FF
:100DD00067204F308A0167204C308A0167204130FC
:100DE0008A01672053308A01672020308A016720FA
:100DF00049308A01672044308A01672045308A01E2
:100E000067204A308A01672045308A016720FE301A
:100E10008A016720C0308A0167204F308A0167202D
:100E200052308A01672041308A0167203A308A01B6
:100E3000672020308A01672020308A016720203017
:100E40008A0167200230A9004208A400A50166308B
:100E5000B000B1018A01B7203A308A016720C8305A
:100E60008A01FB2064008A110A12881B382FC20AEB
:100E70006400183042028A110A12031C402FC2017A
:100E800064008A110A12881A482F8A110A124A2FFE
:100E90008A01072F03170A308D00031342088A01C5
:100EA000ED200A308A01FB20FE308A0167200130E4
:100EB0008A016720FE308A01672080308A0167201E
:100EC00031308A0167202E308A0167204C308A0138
:100ED00067204F308A01672043308A0167205330F2
:100EE0008A0167204F308A0167204C308A016720D1
:100EF00041308A01672053308A01672020308A01FF
:100F0000672049308A01672044308A0167204530D4
:100F10008A0167204A308A01672045308A016720AC
:100F2000FE308A016720C0308A01672050308A0174
:100F3000672045308A01672052308A01672043309C
:100F40008A0167203A308A01672020308A016720B1
:100F500020308A01672020308A0167203A308A01D8
:100F600067200230A9004408A400A5016630B00043
:100F7000B1018A01B720C8308A01FB2064008A11C0
:100F80000A12881BC42FC40A64003C3044028A1130
:100F90000A12031CCC2FC40164008A110A12881A99
:100FA000D42F8A110A12D62F8A01902F03171430DA
:100FB0008D00031344088A01ED200A308A01FB20CA
:100FC000FE308A01672001308A0167200800FE3068
:100FD0008A01672001308A016720FE308A0167207C
:100FE00080308A01672032308A0167202E308A01E2
:100FF000672020308A0167205A308A0167204F30ED
:101000008A0167204E308A01672041308A016720BB
:1010100049308A01672044308A0167204F308A01B5
:1010200067203A308A016720FE308A016720C0308D
:101030008A0167200230A9004D08A400A50166308E
:10104000B000B1018A01B72020308A0167205030FA
:101050008A01672045308A01672052308A01672063
:1010600043308A016720C8308A01FB2064008A155A
:101070000A12881B3C28CD0A640015304D028A15DF
:101080000A12031C4428CD0164008A150A12081AAA
:101090004C288A150A124F288A150A121428031799
:1010A0003C308D0003134D088A01ED200A308A017F
:1010B000FB20FE308A01672001308A016720FE3064
:1010C0008A01672080308A01672032308A016720D8
:1010D0002E308A0167204C308A0167204F308A0108
:1010E000672043308A01672053308A0167204F30E0
:1010F0008A0167204C308A01672041308A016720CD
:1011000053308A01672020308A01672049308A01E4
:10111000672044308A01672045308A0167204A30C1
:101120008A01672045308A016720FE308A016720E6
:10113000C0308A0167204F308A01672052308A010F
:10114000672041308A0167203A308A0167202030C9
:101150008A01672020308A01672020308A016720B9
:101160000230A9004308A400A5016630B000B10117
:101170008A01B7203A308A016720C8308A01FB20F3
:1011800064008A150A12881BC628C30A6400183036
:1011900043028A150A12031CCE28C30164008A1573
:1011A0000A12081AD6288A150A12D9288A150A128C
:1011B0009528031728308D00031343088A01ED207A
:1011C0000A308A01FB20FE308A01672001308A0143
:1011D0006720FE308A01672080308A016720323024
:1011E0008A0167202E308A0167204C308A016720EF
:1011F0004F308A01672043308A01672053308A01CB
:1012000067204F308A0167204C308A0167204130C7
:101210008A01672053308A01672020308A016720C5
:1012200049308A01672044308A01672045308A01AD
:1012300067204A308A01672045308A016720FE30E6
:101240008A016720C0308A01672050308A016720F8
:1012500045308A01672052308A01672043308A0175
:1012600067203A308A01672020308A0167202030C9
:101270008A01672020308A0167203A308A0167207E
:101280000230A9004508A400A5016630B000B101F4
:101290008A01B720C8308A01FB2064008A150A122F
:1012A000881B5329C50A64003C3045028A150A127E
:1012B000031C5B29C50164008A150A12081A6329F8
:1012C0008A150A1266298A150A121F290317323055
:1012D0008D00031345088A01ED200A308A01FB20A6
:1012E000FE308A01672001308A0167200800FE3045
:1012F0008A016720D0308A01672000308A01672088
:101300000715831607118312081483160810FE3080
:1013100083128A016720D3308A01672001308A0155
:1013200067202D308A016720FE308A016720D53082
:101330008A01672002308A0167208A150A126C220E
:10134000081083160810FE3083128A016720D430FB
:101350008A01672020308A01672020308A016720B7
:10136000881483168810FE3083128A016720D330D8
:101370008A01672001308A0167202D308A016720A9
:10138000FE308A016720D5308A01672003308A0148
:1013900067208A150A126C22881083168810FE3086
:1013A00083128A016720D4308A01672020308A01A5
:1013B000672020308A016720081583160811FE3047
:1013C00083128A016720D3308A01672001308A01A5
:1013D00067202D308A016720FE308A016720D530D2
:1013E0008A01672004308A0167208A150A126C225C
:1013F000081183160811FE3083128A016720D43049
:101400008A01672020308A01672020308A01672006
:10141000881583168811FE3083128A016720D33025
:101420008A01672001308A0167202D308A016720F8
:10143000FE308A016720D5308A01672005308A0195
:1014400067208A150A126C22881183168811FE30D3
:1014500083128A016720D3308A01672020308A01F5
:101460006720FE308A016720D4308A01672020304F
:101470008A01672020308A0167200711831607112F
:1014800083120130C10064000B3041028A150A1238
:1014900003186B2AFE308A016720D0308A0167204A
:1014A00000308A0167200130A300F4308A01FC205B
:1014B000FE308A016720D0308A01672020308A01FF
:1014C00067200130A300F4308A01FC20C10A8A158C
:1014D0000A12031D432A08000130CA0064004A08AA
:1014E0004B028A150A12031CC92A0130C10064008C
:1014F0003D3041028A150A120318C42A64008A1575
:101500000A12881BB72A0810831608108312881045
:10151000831688108312081183160811831288110C
:10152000831688118312071183160711FE30831268
:101530008A016720D3308A01672020308A01672022
:10154000FE308A016720D4308A01672020308A016A
:10155000672020308A016720FE308A016720D03062
:101560008A01672020308A0167208A01DB2C8A15D6
:101570000A12CA220330A300E8308A01FC20C10A03
:101580008A150A12031D772ACA0A8A150A12031D30
:101590006E2A08000230BC000730BA001030B800D4
:1015A0000730BB000830B900A2308A011D203C087A
:1015B0008A011D208A010220D0000330BC000730C0
:1015C000BA001030B8000730BB000830B900A230B4
:1015D0008A011D203C088A011D208A010220C900C1
:1015E0000430BC000730BA001030B8000730BB0030
:1015F0000830B900A2308A011D203C088A011D2054
:101600008A010220BF0050184814501C4810D018FE
:10161000C814D01CC81050194815501D4811D019B5
:10162000C815D01DC811501A4014501E4010D01AB1
:10163000C014D01EC010501B4015501F4011D01BAD
:10164000C015D01FC01149184714491C4710C918AC
:10165000C714C91CC71049194715491D4711C91995
:10166000C715C91DC711491A3E14491E3E10C91A93
:10167000BE14C91EBE10491B3E15491F3E11C91B91
:10168000BE15C91FBE113F1846143F1C4610BF1897
:10169000C614BF1CC6103F1946153F1D4611BF1981
:1016A000C615BF1DC6113F1A3D143F1E3D10BF1A7F
:1016B000BD14BF1EBD10FE308A01672080308A0134
:1016C000672049308A01672044308A0167204F3003
:1016D0008A0167203A308A01672020308A0167201A
:1016E00020308A01672020308A01672020308A015B
:1016F0006720A9013D08A400A5016630B000B10132
:101700008A01B720A9014608A400A5016630B000EF
:10171000B1018A01B7203A308A016720A9013E0849
:10172000A400A5016630B000B1018A01B720A9016B
:101730004708A400A5016630B000B1018A01B720B6
:101740003A308A016720A9014008A400A50166304B
:10175000B000B1018A01B720A9014808A400A50181
:101760006630B000B1018A01B7200800FE308A015E
:10177000672001308A016720FE308A0167208030AF
:101780008A0167204F308A01672052308A01672022
:1017900041308A01672020308A01672042308A0167
:1017A000672045308A01672041308A0167204C302C
:1017B0008A0167204C308A01672049308A016720FE
:1017C00054308A01672041308A01672053308A01F2
:1017D00067203A308A0167203D08A600A7010A3039
:1017E000A200A3018A015021B2002508B3004608D7
:1017F0003207CE00FE308A016720C0308A016720A0
:101800004F308A01672052308A01672041308A01B7
:1018100067203A308A01672020308A016720203013
:101820008A01672020308A0167200230A9004E0813
:10183000A400A5016630B000B1018A01B7203A309A
:101840008A016720C8308A01FB2064008A150A12C9
:10185000881B2B2CCE0A640018304E028A150A12FF
:10186000031C332CCE0164008A150A12081B772C46
:101870004E08A000A1010A30A200A3018A01342170
:10188000B2002108B3003208A6003308A7001030C8
:10189000A200A3018A015021B2002508B3004E081E
:1018A000A000A1010A30A200A3018A01342124086A
:1018B000B4002508B50032083407BF000430BC006E
:1018C0000730BA001030B8000730BB000830B9004C
:1018D000A2308A011D203C088A011D203F088A0190
:1018E0001B200A308A01FB208A150A127A2C8A15DD
:1018F0000A12FA2BFE308A01672001308A01672024
:10190000FE308A01672080308A0167204F308A01CB
:10191000672052308A01672041308A0167202030D9
:101920008A01672042308A01672045308A0167209A
:1019300041308A0167204C308A0167204C308A018F
:10194000672049308A01672054308A01672041307E
:101950008A01672053308A0167203A308A01672064
:101960003E08A600A7010A30A200A3018A01502167
:10197000B2002508B30047083207CF00FE308A01C5
:101980006720C0308A01672050308A0167204530C7
:101990008A01672052308A01672043308A0167201C
:1019A0003A308A01672020308A01672020308A017E
:1019B000672020308A0167203A308A016720023090
:1019C000A9004F08A400A5016630B000B1018A014A
:1019D000B720C8308A01FB2064008A150A12881BD0
:1019E000F22CCF0A64003C304F028A150A12031C05
:1019F000FA2CCF0164008A150A12081B3E2D4F08ED
:101A0000A000A1010A30A200A3018A013421B20082
:101A10002108B3003208A6003308A7001030A20046
:101A2000A3018A015021B2002508B3004F08A0008D
:101A3000A1010A30A200A3018A0134212408B400C4
:101A40002508B50032083407C9000330BC00073050
:101A5000BA001030B8000730BB000830B900A2301F
:101A60008A011D203C088A011D2049088A011B208B
:101A70000A308A01FB208A150A12412D8A150A12A2
:101A8000BE2CFE308A01672001308A0167200800E1
:02400E00323F3F
:00000001FF
